:020000040000FA
:1000000083160313810180298B138B1B04289A000C
:10001000030E9B0083010A089C008A0183130408D5
:100020009D009708031D1728051A3328362817083E
:10003000083C031C2328051E9813051A981703195A
:100040003628980C36281708093C031C282836281F
:10005000051E332813178316031306108312031388
:1000600006100B123428980197013728970A8B1035
:100070001D0884001C088A001B0E83009A0E1A0EAD
:10008000090018089900F03C031D492813141311A6
:100090004729131C782813101808123C03195328F9
:1000A0001808593C031993101808583C031D5E2882
:1000B000931D5C2893114729931547291808113C73
:1000C000031D6428131255291808143C031D4729E1
:0400D0009312552909
:1000F000131D862818084A3C031D81282F309800BC
:10010000B62818085A3C0318862847291808613C65
:1001100003189C280E3098021808613C031C932891
:10012000193098079C281808773C03189C28180851
:10013000D23C03191315472903308A00180861239C
:1001400098009808031947291808603C0318562995
:1001500018087A3C031C562918089319B228931CD6
:10016000B628B4289318B628E03E980018089E00D8
:1001700037221808083C031DCC282708031DA703B5
:100180002708141DC428403E803891005A22203090
:100190005C2211085A2247291808093C031DD92856
:1001A0002708263C031CD72820305C22A70A2030D1
:1001B00098002708273C0318DE28A822A70A180859
:1001C0005C221E087A3C031C47291E08403C031889
:1001D000F2289E121E08403C031847291E0D923E2D
:1001E000A10035291E082F3C0318FE281E08393CA3
:1001F000031C28291E0D9F3EA10035291E08223C04
:10020000031D0429483033291E08273C031D0A29F1
:100210004A3033291E08283C031D10294C3033294D
:100220001E08293C031D16294C3033291E082C3C7E
:10023000031D1C294E3033291E082D3C031D222985
:10024000503033291E082E3C031D472952303329D4
:100250001E083A3C031D2E29543033291E083F3C0A
:10026000031D47295630A10035299317A1000330FB
:100270008A0021080723A400A10A21080723A3005C
:100280004729A8220D3037220A303722003483163E
:10029000031306148312031313130B16080093148D
:1002A000003413160034931600344729931CB628E3
:1002B00018080D3C0318B6281908613C031CB62821
:1002C00019083C3C031867293D3099027029190828
:1002D000243C03186E2923309902702904309907B1
:0C02E00003308A001908DA239800B628C1
:1003000005108510851183120313051485108316BB
:100310000313061405160113831203130B1697011A
:10032000930183160313013086058312031386128B
:1003300006138613E130860504302722033053224A
:100340006D2201302722083053226D2201302722EE
:10035000023053226D220130272228305A220C30DD
:100360005A2201305A22083027222830A700F830BC
:100370008B058B172730910002308A001108273C2B
:10038000D8229200372212085C22910BBC290D3032
:1003900037220A3037220A303722FF308C000230F1
:1003A000912290308C0003309122C0308C000330B9
:0C03B0009122131B4120931BE021D9294E
:1003C0002308A5002408A6009313A20102309E0072
:1003D00008309F009E1826089E1C2508A000A01F1C
:1003E000F329A20A0A2AA20803190A2A8514220854
:1003F000013C031C002A91308C0001309122042A18
:10040000FA308C000530912285100630202206300B
:100410002E22A201A00D9F0BEF299E0BE829083088
:08042000202206302E22080004
:100440008C00810183160313C030810508008C00E5
:10045000810183160313C0308105013081048312AA
:1004600003130B110B1D322A8C0B312A0800950047
:10047000051008308C00482215180514151C0510AD
:10048000950C48228C0B3C2A05144822482208006F
:100490001D308D004E2A08308D004E2A8D0B4E2ABD
:1004A0000800960137288E00E13086050E0D1E39B2
:1004B0008604080094145D2A94108F007622941C00
:1004C00086170F080F0E53226D220F0853226D223C
:1004D000E130860586130613080086160000861292
:1004E000080018308E008E0B732A0800861314142F
:1004F000831603131E3086048312031306170000AD
:1005000086167122061E1410861271226D2214188E
:10051000802A061383160313E13086058312031322
:1005200008008D00810183160313073081008312B8
:1005300003130B118515A3228511A3220B1D9A2AE3
:100540008D0B992A08000C088E008E0BA52A080036
:100550002830A700141DB72A80305A2214112030E9
:100560005C22A70BAF2A80305A22A7010800C030B6
:100570005A22141520305C22A70BBA2AC0305A2206
:04058000A7010800C7
:1005B000820750344934433420343134363446349D
:1005C0003834343420344134543420344B3465349A
:1005D000793462346F346134723464342034443496
:1005E000653463346F346434653472342034633476
:1005F0006F346E346E34653463347434653464340B
:02060E00820761
:10061000DB346C34B634D834AD34B034AB346034FD
:10062000AA34C034AA348034D5344034DA34A03407
:10063000DB345034DB346834B0340034D534003427
:10064000D6348034D434003480340034AD340034B3
:10065000DA340034AA340034A0340034B634C03460
:10066000D6340034B5340034D8340034D0340034B7
:10067000DB340034B6348034DA34C034B43400347B
:10068000A8340034C0340034AC340034AB3400340B
:10069000B6340034D5348034D634C034DA348034BF
:1006A000B5346834B634DA34D634D634DA34B634C1
:1006B000D5345834B534AC34DB345434AD34A83488
:0E06C200820700343934003435343334313497
:1006D000323432340034303438343634343409343B
:1006E000A7340034003451294F2900345329713480
:1006F0003134003400340034793473346134773465
:10070000323400340034633478346434653434343F
:100710003334003400342034763466347434723424
:100720003534003400346E346234683467347A34DB
:1007300036340034003400346D346A347534373460
:100740003834003400342C346B3469346F34303432
:100750003934003400342E342D346C34F634703493
:100760002734003400340034E4340034FC345E3484
:100770000034003400344F2941292134003424341A
:100780000034003400343C3430342E3432343534C8
:10079000363438340034003431342B3433342D348F
:1007A0002A343934003408340034003431343734D6
:1007B0003434373482072F34283423342A343B34FA
:1007C0000034003400343D342934003425343A34C4
:1007D0005F3400345C3400343F3440342634003419
:1007E0007B3400345B347E3400342B3400340034EA
:1007F00000345D3400347D340034223400343E341F
:02400E00F13F80
:00000001FF
